:0440000002423D3209
:01400B003282
:01401300327A
:03401B0002405907
:01402300326A
:01402B003262
:0B423D007581101241B4E5826003029D
:02424800403301
:07424A0074004400602974B8
:05425100812400F97456
:05425600423400FA9063
:06425B004281780075A00D
:0D42610000E493F2A308B8000205A0E58276
:0B426E00B501F1E583B502EC75A0FF7F
:05427900E4F50EF50D57
:03427E00024033C8
:0540330012419080FE27
:0E40380075A888758920758B64758D647588F0
:0D404600409041B0E493FA908000E0FB90C0
:054053008000EA5BF0B3
:014058002245
:0E405900C0E0C0F0C082C083C002C003C0D06F
:0E40670075D000908000E0FA53020FBA0E1CD4
:0D40750090FFFFE4F0740F550C44D054DFB1
:0D408200F50C908000F090FFFF7480F002BC
:02408F004101ED
:0B409100908000E0FA53020FBA0B1BF6
:0D409C0090FFFFE4F0740F550C4470547F4A
:0D40A900F50C908000F090FFFF7480F08017
:0140B6004ABF
:0B40B700908000E0FA53020FBA0D1BCE
:0D40C20090FFFFE4F0740F550C44E054EF44
:0D40CF00F50C908000F090FFFF7480F080F1
:0140DC0024BF
:0B40DD00908000E0FA53020FBA0719B0
:0D40E80090FFFFE4F0740F550C44B054BF7E
:0C40F500F50C908000F090FFFF7480F04C
:0E410100908000E0FA5302F09041ACE493FB92
:04410F00EAB5030604
:0641130090FFFF745FF055
:0E411900908000E0FA5302F09041ADE493FB79
:04412700EAB50306EC
:06412B0090FFFF7444F058
:0E413100908000E0FA5302F09041AEE493FB60
:04413F00EAB50306D4
:0641430090FFFF743EF046
:0E414900908000E0FA5302F09041AFE493FB47
:04415700EAB50306BC
:06415B0090FFFF7476F0F6
:0B4161007401250DFAE4350EFBE4F5B7
:09416C0010750F048A828B831286
:0B4175004205E5828583F0F50D85F022
:014180000E30
:0E418100D0D0D003D002D083D082D0F0D0E0D6
:01418F0032FD
:0B419000124038759850758780C29966
:02419B0080FEA4
:01419D0022FF
:0A419E005F443E7665737B467F7731
:0441A800D0E070B043
:0441AC00D0E070B03F
:0441B000FDFEF7FB1E
:0341B40075820011
:0141B70022E5
:0841B800E50F451060467A0195
:0741C000E50F25E0F50FE516
:0941C70010334012F510E5829559
:0A41D0000FE583951040030A80E616
:0341DA00C3E5102A
:0741DD0013F510E50F13F5C7
:0141E4000FCB
:0C41E500C3E582950FF5F0E583951040CE
:0641F10005F58385F08254
:0741F700C3E51013F510E50C
:0641FE000F13F50FDAE1DA
:014204002297
:0E420500C2D5E58330E70DD2D5E4C39582F52E
:0642130082E49583F583AF
:0C421900E51030E70DB2D5E4C3950FF5B9
:054225000FE49510F507
:01422A001083
:0E422B001241B830D50BE4C39582F582E495BC
:0342390083F58387
:01423C00225F
:00000001FF
